:020000020000FC
:1000000010C0189518951895189518951895189565
:1000100018951895D0C118951895BDC118951895C3
:10002000F3C10FEF0DBF04E00EBFAA240FE30AB91E
:1000300000E40BB908E308B90EE207B90DE005B911
:1000400002E004B981D297D2BCD200E49CD2E4E8A9
:10005000F6E09DD2A0928000A092810004E005BD50
:1000600001E000936E0004E000BF789469D131F0A4
:10007000E4E0F6E084D28BD29DD27DD209E1D02E8D
:100080009F7797FD53C0DD20E1F7EE20D1F7D9F738
:100090000DE7E02EA3D060F44398A0D048F40DE71C
:1000A000E02E439A459A9AD018F4439A459896D0F0
:1000B000349B3CC01B9B07C0C1D0D7D0F1D035D1F9
:1000C000439A459ADBCFF894A0926E00A0926F00FD
:1000D000A0BE02EE0093800009E100938100A0928F
:1000E00089000CE300938800A092870008E7009342
:1000F000860000E448D2EEEEF5E049D2789400ECB8
:10010000C8D10FEF13E02017310741F0022F132F52
:10011000E7D1A8D156D21B9998CFF1CF05E433D2BD
:10012000ECE7F6E034D21B9990CFE9CF04E052D04F
:10013000189B0FC01A9B01C03AC043984FD0439AF6
:1001400040E050E068EE73E0A0E0B0E0EBE0F1E00A
:100150000AC044D073D040E050E060E177E2A0E014
:10016000B0E0E9E0F1E0002411242224332480E30C
:10017000440F551F661F771FAA1FBB1F001C111CB1
:10018000221C331C001611062206330628F0001A22
:10019000110A220A330A43958A9551F7672B6A2B75
:1001A0006B2B81F440835183BAD0DCD067CF16D05B
:1001B000232B41F4373030F400930D0110930E01DE
:1001C000AED05CCFDCD1E4EFF5E0E1D10AEF02D0B4
:1001D000D2D154CFD02EDD20F1F70895419AF1D13C
:1001E0004198A0928500A0928400222404E1439BC0
:1001F00008E9459B08E9302E01E206BB01E20093C5
:100200006F0001E000936E00987F01E4009381008D
:10021000569892FD0BC091FFFCCF00E40093810043
:10022000042D152D262D372D8894089500E4009374
:10023000810004E0CFDF3FEF08940895439B14C092
:10024000459B12C040910D0150910E01041B150BEE
:100250002A093A0948F49160009510952095309547
:100260000A1D1A1D2A1D3A1D0895C9E0D1E0439BBD
:100270002296459B229668817981441B550B81E229
:1002800010F4460F571F57954795379527951795A3
:1002900007958A95A9F7022F132F242F352F08953C
:1002A000AFE0B1E066276395442750E2000F111FCD
:1002B000221F331F441F4A3010F04A5003955A95AD
:1002C000A9F74D930A151A052A053A0561F7623018
:1002D00010F4AD926395439B6D5F459B6C5FEEE0C0
:1002E000F6E090FF369636966A956230E0F7112771
:1002F000C1E0D1E0C8953196002DE894002311F4B7
:1003000000FB0E91FF93EF93E8E6F6E0E00FF11F9C
:10031000C895EF91FF910992C73061F70895C1E048
:10032000D1E0A992C730E9F7089529D1E8EEF5E0C8
:100330002ED1E1E0F1E00191E8D0E730E1F7089556
:10034000C9E0D1E040E050E021D00993500FCD301A
:10035000D9F71CD0051729F00FEF0A930A930A93D7
:100360000A930895C9E0D1E040E050E00991500FB0
:1003700003D0CD30D9F7052F41BD439500BDF8948A
:10038000FA9AF99A7894F999FECF089541BD439568
:10039000F89A00B508950F930FB70F932394231481
:1003A00028F03A9A569A946001E000936E000F91FB
:1003B0000FBF0F9118950F930FB70F933A9B0CC077
:1003C0004090860050908700622C3A9804E10A958C
:1003D000F1F700E206BB14C0742C40908600471869
:1003E000752C509087005708762C622C670877246C
:1003F0003A9A569A01E000936E00A0926F009260C4
:100400000F910FBF0F9118950F9309ED06BD7894CA
:100410000FB71F930F93FF93EF93E0E0F1E010818C
:100420001395143010F009D011271193EF91FF911B
:100430000F911F910FBF0F91189506B1087000958D
:10044000007110850087011731F417810783102789
:10045000102309F09068DD2009F0DA94EE2009F00D
:10046000EA9408950F931F932F9300E48CD0EEEE3F
:10047000F5E08DD0032F49D00F9147D00CE245D045
:100480000F9143D00F9141D000E23FD004EF3DD017
:10049000089500937C0083D022273327442703EC60
:1004A00000937A0000917A0006FDFCCF112703EC3F
:1004B00000937A0000917A0006FDFCCF009178004D
:1004C000200F00917900301F4A1D1A9581F72038BE
:1004D00010F03F5F4F4F232F342FA0927A000895E2
:1004E0004FE2439500511742E0F73AE33A9508513D
:1004F0001C4FE0F32FE2239504561040E0F71AE377
:100500001A95065FE8F3005D08950F9302950F704A
:1005100000610BB913D00F910F7000610BB90ED0B1
:1005200057D008955C980F9302950F700BB906D0C1
:100530000F910F700BB902D04BD008955D9A000057
:10054000000000005D98089506E029D00A95E9F7BB
:1005500003E00BB9F3DF23D0F1DF21D0EFDF1FD0B1
:1005600002E00BB9EBDF1BD008E2DCDF0CE0DADFE6
:1005700004E0D8DF089501E0D5DF11D0089502E04E
:10058000D1DF0DD008950068CDDF09D00895C8955A
:10059000002021F0002DB9DF3196F9CF08950F9397
:1005A0001F9302E519EC1A95F1F70A95D9F71F91F7
:1005B0000F9108950F9309E004D00A95E9F70F9180
:1005C00008950F9303E1EBDF0A95E9F70F91089582
:1005D0000F9306EA0A95F1F70F9108952020202045
:1005E00020202020202020004361703A2000455325
:1005F000523A20004B616C696272696572756E6770
:1006000021202000454550524F4D2D4665686C65B0
:10061000722120000A0010000D110010000F0D11B2
:10062000000010000D110F0000000D11001000005F
:100630000C11000010000C110F0000000C11001034
:1006400000000B11000010000B110F0000000B1137
:10065000000000000B110F13120F0F0F0F13120FDA
:100660000F0F0F13120F0F0F30313233343536376F
:1006700038392DE46EE645202C464C4F4F4C202057
:10068000202020002020202020202020202020208A
:02069000200048
:00000001FF
